S01400006F7064726163687420332E332E7372656307
S113000045C0000060C000005EC000005CC000008D
S11300105AC0000058C0000056C0000054C0000080
S113002052C0000069C000004EC000004CC0000077
S11300304AC0000048C0000046C0000044C00000A0
S113004042C0000040C000003EC000003CC00000B0
S11300503AC0000038C0000036C0000034C00000C0
S113006032C0000030C000002EC000002CC00000D0
S11300702AC0000028C0000026C0000024C00000E0
S113008022C0000020C000001EC0000011241FBEBA
S1130090CFEFD0E1DEBFCDBF11E0A0E0B1E0E2E4FC
S11300A0F1E000E00BBF02C007900D92A030B10751
S11300B0D9F721E0A0E0B1E001C01D92A030B20761
S11300C0E1F734D03CC09CCF20E030E008C0E3EC42
S11300D0F9E03197F1F700C000002F5F3F4F281778
S11300E03907ACF3089586E983BD87B7806887BF75
S11300F078948DE085BD08951F920F920FB60F92EC
S113010011248F939F9395B381E0892785BB83B591
S11301108A3F19F486E983BD02C08AEF83BD9F91AB
S11301208F910F900FBE0F901F9018958FEF84BB87
S113013081E085BBD8DF8AE090E0C6DFFCCFF8948D
S1050140FFCFEB
S9030000FC
